:10000000073099007B202C288B13B700030EB80013
:100010000A08B900051C0D2818280930850536186E
:100020008516B618051636190515B6198514232830
:1000300009308505361A8516B61A0516361B0515BC
:10004000B61B851423280B1039088A00380E83004C
:10005000B70E370E8B1709001030BA00BC01BB0178
:1000600063203F080310BC070318BB0ABA0B3028F3
:10007000A7013B08A6003C08A5008D207D30AF00FD
:100080002030AE00AD01AC0164218830AF00AA3051
:10009000AE00AD01AC01CF217C30AF003830AE00F6
:1000A0005130AD00EC30AC0064218530AF00103031
:1000B000AE00AD01AC01CF210921A71F6028A50129
:1000C0002508B6002C282030BE003630BD00C00107
:1000D000BF01031100008519C00A0319BF0ABE0B36
:1000E0006A28BD0B6B280310C00DBF0DC00DBF0DDE
:1000F000C00DBF0D080083169F01FF2390308512AD
:1001000005120511851016148B1583128512051220
:10011000051185100B108B1708009630A800A90157
:10012000A71F9B28A509A609A709A50A0319A60ABE
:100130000319A70AA917B3012708031DB028260829
:10014000A7002508A600A501B3152708031DB028A0
:100150002608A700A601B311331627080319C128E2
:100160003308A802031D031CC2290310A71BBE28C5
:10017000A50DA60DA70DA80BB628C229A91FA71368
:100180000034A701A601A501A401A8010034B30110
:100190002708031DE7282608A7002508A60024082D
:1001A000A500A401B3152708031DE7282608A7000A
:1001B0002508A600A501B31133162708031DE7285B
:1001C0002608A700A601B31527080319C12833087C
:1001D000A802031D031CC2290310A71BF628A40DA7
:1001E000A50DA60DA70DA80BED28C2292A1B251CBD
:1001F000BE28A41FBE28A50A0319A60A0319A70A28
:10020000031DBE28A70CA60CA50CA80A0319B72924
:10021000BE282808031900342708A900A71796301C
:10022000A802A81F5829A809A80A08302802031CF8
:100230003429A800A50D2608A5002708A600A701B7
:1002400008302802031C3429A800A50D2608A500A3
:10025000A60108302802031C3429A800A50DA50119
:100260002808031D03103D29280803193D29031000
:10027000A70CA60CA50CA80B37292A1B251C49295D
:10028000031C4929A50A0319A60A0319A70AA71BD3
:100290005829A91F0034A709A609A509A50A031909
:1002A000A60A0319A70A0034A701A601A501003474
:1002B0002A14AA1FFF34A701A91FFF30A700A60018
:1002C000A500A90DA70CFF342808031D2F0803194A
:1002D000C12827082E06A9002F08A8077E30031C76
:1002E0007529A8020318B7297829A802031CC22976
:1002F0002708A4002608A3002508A200A417AE170B
:100300000310A701A601A5011830B300221C9229F1
:100310002C08A5072D0803182D0FA6072E08031873
:100320002E0FA707A70CA60CA50CA40CA30CA20CBF
:100330000310B30B8629A71BA229A40DA50DA60D9A
:10034000A70DA8032A1B251CB429A41FB429A50A9C
:100350000319A60A0319A70A031DB429A70CA60CA2
:10036000A50CA80A0319B729A91FA7130034AA14BA
:10037000AA1FFF34FF30A800A700A600A500A90D02
:10038000A70CFF342A15AA1FFF340130A800A701CB
:10039000A601A501A90DA70CFF348030AE062708E1
:1003A0002E06B300A401AB0128082F02031CF0297C
:1003B0002F08A2002808AF002208A8002E08A200DB
:1003C0002708AE002208A7002D08A2002608AD00CD
:1003D0002208A6002C08A2002508AC002208A500CF
:1003E0002F08031900342708A900A717AE172F08F4
:1003F0002802AF000319232A08302F02031C192AF0
:10040000AF002C08AB002D08AC002E08AD00AE01EB
:1004100008302F02031C192AAF002C08AB002D084E
:10042000AC00AD0108302F02031C192A2908A700CF
:1004300000342F080319232A0310AE0CAD0CAC0CAA
:10044000AB0CAF0B1C2AB31F302AAB09AC09AD09AA
:10045000AE09AB0A0319AC0A0319AD0A0319AE0AB7
:100460002B08A4072C0803182C0FA5072D08031828
:100470002D0FA6072E0803182E0FA707B31B492A16
:10048000031CF628A70CA60CA50CA40CA80FF62894
:10049000B7290318C728A409A509A609A709A40A0A
:1004A0000319A50A0319A60A0319A70A8030A90689
:1004B0009B288400AE010A30AD006622220880002D
:1004C000303080078403B50B5A2A0800A301A2012B
:1004D0001030B400270DA20DA30D2D08A2022E0886
:1004E000031C2E0FA30203187C2A2D08A2072E0836
:1004F00003182E0FA3070310A60DA70DB40B6A2A2D
:020500000034C5
:02400E0084111B
:00000001FF
